:020000040000FA
:0600000050EF12F01200A7
:020006001200E6
:0600080015EF01F01200EB
:02000E000100EF
:0C001000BC24000000010000B90000004A
:04001C00D9CFE6FF53
:10002000E1CFD9FFFB0EDBCF1DF0FC0EDBCF1EF0C6
:10003000FD0EDBCF1FF0FE0EDBCF20F02034000ED4
:10004000201809E6D880000E1D54000E1E54000E24
:100050001F54000E20540CE2D950FB0FE96EFF0E26
:10006000DA20EA6EEE06000EEE5AEE5AEE5ADAD7B3
:10007000E552E7CFD9FF1200948E949C200EAF6E0C
:10008000AC8AAC84AC98AC9CAB8EAB9CAB889E9895
:100090009E9A9D8AF28EF28C1200D9CFE6FFE1CFB4
:1000A000D9FFE65200018751851902E1885186196E
:1000B00001E1F8D785C0E9FF86C0EAFF852B000E75
:1000C0008623EFCFDFFF930E855D010E865904E393
:1000D000530E856F010E866FDF5000D0E552E5525A
:1000E000E7CFD9FF1200D9CFE6FFE1CFD9FF020E4B
:1000F000E126DE6ADD6AACB210D0DF2A010E01E330
:10010000DB2AD9CFE9FFDACFEAFF100ED880EE5410
:10011000270EED5401E206D0EED7FE0EDB50AD6E99
:100120009EA8FED7020EE15C02E2E16AE552E16EB2
:10013000E552E7CFD9FF1200D9CFE6FFE1CFD9FFD3
:10014000030EE126FD0EDBCFDEFFDBCFDDFFA5DFFB
:10015000E76E020EE7CFDBFFFC0EDB50F36E020E04
:10016000DB50F35C0DE0FD0EDBCFE9FFDB2AFE0E7A
:10017000DBCFEAFF01E3DB2A020EDBCFEFFFE7D79D
:10018000FD0EDBCFE9FFFE0EDBCFEAFFEF6ADECF2D
:1001900000F0DDCF01F000C0F3FF01C0F4FF030E5B
:1001A000E15C03E200D0E16AE552E16EE552E7CF9F
:1001B000D9FF1200D9CFE6FFE1CFD9FF020EE12629
:1001C000DE6ADD6AFD0EDBCFE9FFFE0EDBCFEAFF64
:1001D000EF5014E0FD0EDBCFE9FFFE0EDBCFEAFFB0
:1001E000EF50E66E80DFE552DF2A010E01E3DB2AE5
:1001F000FD0EDB2AFE0E01E3DB2AE4D7010EF36ECF
:10020000F46A020EE15C03E200D0E16AE552E16EBD
:10021000E552E7CFD9FF12000D0EE66E64DFE5521E
:100220000A0EE66E60DFE5521200DACFE4FFE2CF9D
:10023000DAFFE9CFE4FFEACFE4FFF6CFE4FFF7CF40
:10024000E4FFF5CFE4FFF3CFE4FFF4CFE4FFFACF10
:10025000E4FF00EE18F0140EE80403E3EECFE4FF31
:10026000FBD700EE00F0180EE80403E3EECFE4FF46
:10027000FBD7E6529EAA4DD0D2EC11F00001D36F0D
:10028000AB50040B03E1AB50020B02E0AB98AB8820
:10029000ACA2FED781B205D0D3C0E6FF29EC12F0A4
:1002A000E552080E0001D35D0DE1000EE76ED21994
:1002B000E8AE02D0D23503D0E750D880D25501E263
:1002C000D20727D00D0ED35D17E0400EE76ED2198E
:1002D000E8AE02D0E73402D0E750D25D0DE2D25151
:1002E000D22BE96EEA6AE9BEEA68530EE926010EEE
:1002F000EA22D3C0EFFF0DD0D2C0E9FFEA6AE9BE1F
:10030000EA68530EE926010EEA22EF6AD26B010E6B
:10031000846F9EA40AD0BECFAAF0BFCFABF000017D
:10032000AC6BAD6B9785CD909E94E55200EE17F0C7
:10033000180EE80403E3E5CFEDFFFBD700EE2BF04A
:10034000140EE80403E3E5CFEDFFFBD7E5CFFAFF9A
:10035000E5CFF4FFE5CFF3FFE5CFF5FFE5CFF7FFFE
:10036000E5CFF6FFE5CFEAFFE5CFE9FFE5CFDAFF1E
:100370001100D9CFE6FFE1CFD9FF0A0EE126000137
:10038000420E826F010E836FFC0EDBCF00F0010E78
:10039000E76E0018E8AE02D0003403D0E750D880F2
:1003A000005401E2DBD0FC0EDB5028E1FD0EDBCF78
:1003B00000F0FE0EDBCF01F0060E00C0DBFF070EE3
:1003C00001C0DBFF080EDB6A090EDB6A82C0E6FFB4
:1003D00083C0E6FFD950060FE96EDACFEAFFEECF11
:1003E000E6FFEECFE6FFEECFE6FFEFCFE6FF6FECE6
:1003F0000FF0006E060EE15E005010D082C0E6FFE6
:1004000083C0E6FFFD0EDBCFE6FFFE0EDBCFE6FF8F
:10041000D5EC0EF0E552E552E552E552000197ADFC
:1004200084D0420EE66E010EE66EA0EC11F0E552AD
:10043000E552020EF3CFDBFF030EF4CFDBFFDE6AE3
:10044000DD6ADECF00F0DDCF01F0020EDBCF02F07F
:10045000030EDBCF03F00250005C035001582EE284
:10046000020EDBCF02F0030EDBCF03F0DE50025CA6
:10047000E96EDD500358EA6EE906000EEA5A420EB4
:10048000E926010EEA22EF50E66EFC0EDB50040F67
:10049000006E016A00BE0168DE50005CE96EDD504E
:1004A0000158EA6E420EE926010EEA22E552E750B3
:1004B000EF6EDF2A010E01E3DB2AC3D7DE6ADD6AB5
:1004C000DECF00F0DDCF01F0FC0EDB50050F046E37
:1004D000056A04BE0568020EDB50045C026E030E62
:1004E000DB500558036E0250005C035001581DE2BA
:1004F000000197A90BD0DECFE9FFDDCFEAFF420E66
:10050000E926010EEA22300EEF6E0AD0DECFE9FFB7
:10051000DDCFEAFF420EE926010EEA22200EEF6E41
:10052000DF2A010E01E3DB2ACBD7FC0EDB50050FDF
:10053000E96EEA6AE9BEEA68420EE926010EEA229D
:10054000EF6A82C0E6FF83C0E6FF34DEE552E55283
:10055000020EF3CFDBFF030EF4CFDBFF0A0EE15CEC
:1005600002E2E16AE552E16EE552E7CFD9FF1200FF
:10057000D9CFE6FFE1CFD9FF0C0EE126F80EDBCF95
:1005800002F0000EE76E0218E8AE02D0023403D08B
:10059000E750D880025402E3070E12D0F80EDBCFEA
:1005A00003F0160EE76E0318E8AE02D0033403D052
:1005B000E750D880035402E2170E02D0F80EDB2871
:1005C000006E016A00BE0168060E00C0DBFF070E68
:1005D00001C0DBFFDE6ADD6AFB0EDBCF00F0FC0E44
:1005E000DBCF01F0FD0EDBCF02F0FE0EDBCF03F020
:1005F000226A236A246A256A00C01DF001C01EF029
:1006000002C01FF003C020F0F1EC0DF0010A33E14D
:10061000F90EDBCFE9FFDB2AFA0EDBCFEAFF01E3BD
:10062000DB2A2D0EEF6EFB0EDBCF00F0FC0EDBCFD6
:1006300001F0FD0EDBCF02F0FE0EDBCF03F0226AED
:10064000236A800E246EBF0E256E00C01DF001C00F
:100650001EF002C01FF003C020F015EC0DF0FB0EE1
:100660001DC0DBFFFC0E1EC0DBFFFD0E1FC0DBFF4D
:10067000FE0E20C0DBFFFB0EDBCF00F0FC0EDBCF5D
:1006800001F0FD0EDBCF02F0FE0EDBCF03F0226A9D
:10069000236A246A256A00C01DF001C01EF002C052
:1006A0001FF003C020F0E8EC0DF0010A49E1FB0E59
:1006B000DBCF00F0FC0EDBCF01F0FD0EDBCF02F054
:1006C000FE0EDBCF03F0226A236A800E246E3F0EFB
:1006D000256E00C01DF001C01EF002C01FF003C057
:1006E00020F0F1EC0DF0010A2BE1006A016A200E06
:1006F000026E410E036ED950FB0FE96EFF0EDA2039
:10070000EA6EEECF1DF0EECF1EF0EECF1FF0EFCF72
:1007100020F000C022F001C023F002C024F003C08A
:1007200025F015EC0DF020C0EDFF1FC0EDFF1EC041
:10073000EDFF1DC0EFFFDF06010E01E2DB06B7D7BC
:10074000FB0EDBCF00F0FC0EDBCF01F0FD0EDBCFAC
:1007500002F0FE0EDBCF03F0226A236A200E246E25
:10076000410E256E00C01DF001C01EF002C01FF03A
:1007700003C020F0F1EC0DF0010A2DE0FB0EDBCF01
:1007800000F0FC0EDBCF01F0FD0EDBCF02F0FE0E21
:10079000DBCF03F0226A236A200E246E410E256E01
:1007A00000C01DF001C01EF002C01FF003C020F009
:1007B000C2EC0CF0FB0E1DC0DBFFFC0E1EC0DBFF0D
:1007C000FD0E1FC0DBFFFE0E20C0DBFFDF2A010E87
:1007D00001E3DB2AB5D7DECF00F0DDCF01F0D95041
:1007E000060FE96EDACFEAFF0050EE260150ED2247
:1007F000010EF36E020EF3CFDBFF030EDB6A020E77
:10080000DBCF1EF0030EDBCF1FF0FDEC0BF0080E6C
:100810001DC0DBFF090E1EC0DBFF0A0E1FC0DBFF81
:100820000B0E20C0DBFF020EDBCF00F0030EDBCF90
:1008300001F0060EDBCF02F0070EDBCF03F0015014
:100840000318E8AE02D0033404D00250005C035019
:1008500001582EE2080EDBCF00F0090EDBCF01F0CD
:100860000A0EDBCF02F00B0EDBCF03F0226A236A05
:10087000200E246E410E256E00C01DF001C01EF03A
:1008800002C01FF003C020F0C2EC0CF0080E1DC027
:10089000DBFF090E1EC0DBFF0A0E1FC0DBFF0B0EC5
:1008A00020C0DBFF020EDB2A030E01E3DB2ABBD7ED
:1008B000080EDBCF04F0090EDBCF05F00A0EDBCF0C
:1008C00006F00B0EDBCF07F0226A236A246A400E83
:1008D000256E04C01DF005C01EF006C01FF007C045
:1008E00020F0C2EC0CF01DC000F01EC001F01FC0D3
:1008F00002F020C003F0D950FB0FE96EFF0EDA20A2
:10090000EA6EEECF1DF0EECF1EF0EECF1FF0EFCF70
:1009100020F000C022F001C023F002C024F003C088
:1009200025F02CEC0CF020C0EDFF1FC0EDFF1EC029
:10093000EDFF1DC0EFFFFB0EDBCF00F0FC0EDBCFA9
:1009400001F0FD0EDBCF02F0FE0EDBCF03F0226ADA
:10095000236A200E246E410E256E00C01DF001C0DA
:100960001EF002C01FF003C020F0F1EC0DF0010AF0
:1009700012E0FB0EDB6AFC0EDB6A800EF36EFD0EEE
:10098000F3CFDBFF3F0EF36EFE0EF3CFDBFFDF2A6C
:10099000010E01E3DB2ADECF00F0DDCF01F0000124
:1009A000800E011459E0F90EDBCFE9FFDB2AFA0EC5
:1009B000DBCFEAFF01E3DB2A300EEF6EF90EDBCF6F
:1009C000E9FFDB2AFA0EDBCFEAFF01E3DB2A2E0E7A
:1009D000EF6E060EDBCF00F0070EDBCF01F0800ECE
:1009E000011410E0DECF02F0DDCF03F0060EDB5085
:1009F000025C006E070EDB500358016E00C0DEFF84
:100A000001C0DDFF020EDB68030EDB68020EDBCFE8
:100A100000F0030EDBCF01F0DECF02F0DDCF03F0FC
:100A200003500118E8AE02D0013404D00050025C3B
:100A30000150035811E2F90EDBCFE9FFDB2AFA0E71
:100A4000DBCFEAFF01E3DB2A300EEF6E020EDB069E
:100A5000030E01E2DB06DAD7020EDB6A030EDB6A65
:100A6000020EDBCF00F0030EDBCF01F0060EDBCF72
:100A700002F0070EDBCF03F001500318E8AE02D0FE
:100A8000033404D00250005C0350015801E3ABD0A2
:100A9000FB0EDBCF1DF0FC0EDBCF1EF0FD0EDBCF1F
:100AA0001FF0FE0EDBCF20F082EC0DF0040E1EC016
:100AB000DBFF050E1FC0DBFF300EE76E040EDBCF41
:100AC00000F0050EDBCF01F0E7500026000E0122FA
:100AD000F90EDBCFE9FFDB2AFA0EDBCFEAFF01E3F9
:100AE000DB2A00C0EFFF020EDBCF00F0030EDBCFEE
:100AF00001F0DF50001803E1DE52DD5001180BE178
:100B0000F90EDBCFE9FFDB2AFA0EDBCFEAFF01E3C8
:100B1000DB2A2E0EEF6E040EDBCF1EF0050EDBCFB0
:100B20001FF0FDEC0BF0080E1DC0DBFF090E1EC010
:100B3000DBFF0A0E1FC0DBFF0B0E20C0DBFF1DC05A
:100B400000F01EC001F01FC002F020C003F0D95019
:100B5000FB0FE96EFF0EDA20EA6EEECF1DF0EECF4E
:100B60001EF0EECF1FF0EFCF20F000C022F001C04A
:100B700023F002C024F003C025F02BEC0CF020C0C1
:100B8000EDFF1FC0EDFF1EC0EDFF1DC0EFFF006AAF
:100B9000016A200E026E410E036ED950FB0FE96E02
:100BA000FF0EDA20EA6EEECF1DF0EECF1EF0EECF94
:100BB0001FF0EFCF20F000C022F001C023F002C0F0
:100BC00024F003C025F015EC0DF020C0EDFF1FC090
:100BD000EDFF1EC0EDFF1DC0EFFF020EDB2A030E6E
:100BE00001E3DB2A3DD7F90EDBCFE9FFFA0EDBCFBD
:100BF000EAFFEF6A0C0EE15C02E2E16AE552E16EA7
:100C0000E552E7CFD9FF1200D9CFE6FFE1CFD9FFF8
:100C1000060EE1260001979DFB0EDBCF1DF0FC0EBA
:100C2000DBCF1EF0FD0EDBCF1FF0FE0EDBCF20F082
:100C3000B1EC0DF01CC0DEFF1DC0DEFF1EC0DEFFEC
:100C40001FC0DDFFDD52DD52FB0EDBCF04F0FC0EDA
:100C5000DBCF05F0FD0EDBCF06F0FE0EDBCF07F09D
:100C6000F90EDBCF1EF0FA0EDBCF1FF0FDEC0BF020
:100C70001DC008F01EC009F01FC00AF020C00BF014
:100C800008C022F009C023F00AC024F00BC025F0F0
:100C900004C01DF005C01EF006C01FF007C020F004
:100CA00015EC0DF01DC000F01EC001F01FC002F0D9
:100CB00020C003F0F90EDBCF14F0FA0EDBCF15F0F5
:100CC000166A176A15AE02D01668176814C01CF0B1
:100CD00015C01DF016C01EF017C01FF0DFCF21F0A9
:100CE000010EDBCF22F0020EDBCF23F0030EDBCFB1
:100CF00024F04FEC11F018C010F019C011F01AC018
:100D000012F01BC013F010C01CF011C01DF012C077
:100D10001EF013C01FF012EC0CF01DC00CF01EC032
:100D20000DF01FC00EF020C00FF00CC022F00DC05F
:100D300023F00EC024F00FC025F000C01DF001C04C
:100D40001EF002C01FF003C020F02BEC0CF082EC70
:100D50000DF0040E1EC0DBFF050E1FC0DBFF000EF2
:100D6000E66E010EE66ED9CFE9FFDACFEAFFEECFED
:100D7000E6FFEECFE6FFEECFE6FFEFCFE6FF6FEC4C
:100D80000FF0006E060EE15E0050000EE66E010EE2
:100D9000E66EDAEC00F0E552E552F3CFA4F0F4CFC2
:100DA000A5F02E0EE66E73EC00F0E552F80EDBCFE8
:100DB000E6FFE66A040EDBCFE6FF050EDBCFE6FFBB
:100DC000B9EC01F0E552E552E552E552060EE15C60
:100DD00002E2E16AE552E16EE552E7CFD9FF120087
:100DE000D9CFE6FFE1CFD9FFE652800EDF6EDF50AC
:100DF000000813E2FE0EDB50DF1406E0310EE66E53
:100E000073EC00F0E55205D0300EE66E73EC00F0A6
:100E1000E552DF407F0BDF6EEAD7E552E552E7CFC0
:100E2000D9FF1200D9CFE6FFE1CFD9FF020EE126AC
:100E3000FE0EDB50F00BE8380F0B300FDF6EDF508B
:100E4000390803E2070EDF24DF6EFE0EDB500F0BC6
:100E5000300FE76E010EE7CFDBFFDB5039080AE207
:100E6000070E006E010EDBCFE7FF0050E726010EF4
:100E7000E7CFDBFFDFCFE6FF73EC00F0E552010EBA
:100E8000DBCFE6FF73EC00F0E552680EE66E73EC24
:100E900000F0E552020EE15C02E2E16AE552E16E29
:100EA000E552E7CFD9FF120081689368938093825F
:100EB000938493869388938A938C938EC26A070E49
:100EC000C16E926E1F0E896E8268860E946E94902B
:100ED0009492948494969498949A949C948E1200EC
:100EE0000001BA6BBB6BBC6BBD6B000EE66EE66AB5
:100EF0000DEC12F0E552E552898689968986CD80FF
:100F00009EA005D00001BC2B000EBD239E9081B099
:100F1000F7D7CD901200C8DF89863CEC00F00001C5
:100F2000979F0C0EE66E73EC00F0E552F00EE66E45
:100F3000490EE66E020EE66EE66A0EEC00F0E55231
:100F4000E552E552E55295C100F096C101F0026A02
:100F500000C0E6FF01C0E6FF02C0E6FF40C1E6FFB9
:100F600041C1E6FF87EC11F0036E050EE15E035010
:100F700040C1E6FF41C1E6FFDAEC00F0E552E55280
:100F8000F3CFA4F0F4CFA5F097C100F098C101F021
:100F9000026A00C0E6FF01C0E6FF02C0E6FF40C1F2
:100FA000E6FF41C1E6FF87EC11F0036E050EE15E3E
:100FB000035040C1E6FF41C1E6FFDAEC00F0E55224
:100FC000E552F3CFA4F0F4CFA5F099C100F09AC197
:100FD00001F0026A00C0E6FF01C0E6FF02C0E6FFC2
:100FE00040C1E6FF41C1E6FF87EC11F0036E050E3C
:100FF000E15E035040C1E6FF41C1E6FFDAEC00F0DC
:10100000E552E552F3CFA4F0F4CFA5F0A00EE66EC2
:10101000860EE66E010EE66EE66A0EEC00F0E55214
:10102000E552E552E552CD6ACD8ECD9ACD98CD965A
:10103000CD84CD92CD909F80000EE66EE66A0DECD9
:1010400012F0E552E5529E90F28C9D90F29EF29C39
:101050009484B19C040EBD6ED08E9D84F28E40DFD0
:10106000000197A510D0AA0EE96E000EEA6EBA51E3
:10107000EE24BA6FBB51EE20BB6FBC51EE20BC6FAB
:10108000BD51EE20BD6FD880220EBA55010EBB5562
:10109000000EBC55000EBD5509E3180EBA5D010ED9
:1010A000BB59000EBC59000EBD5916E29DC100F09F
:1010B0009EC101F0026A00C0E6FF01C0E6FF02C067
:1010C000E6FF40C1E6FF41C1E6FF87EC11F0036E89
:1010D000050EE15E035015D09BC100F09CC101F0EC
:1010E000026A00C0E6FF01C0E6FF02C0E6FF40C1A1
:1010F000E6FF41C1E6FF87EC11F0036E050EE15EED
:101100000350000EE66E010EE66EDAEC00F0E552DA
:10111000E552F3CFA4F0F4CFA5F0090EE66E73EC20
:1011200000F0E552000EE66E010EE66EBAC0E6FF74
:10113000BBC0E6FFBCC0E6FFBDC0E6FF6FEC0FF032
:10114000006E060EE15E0050000EE66E010EE66EC9
:10115000DAEC00F0E552E552F3CFA4F0F4CFA5F0BD
:101160000CEC01F09FC100F0A0C101F0026A00C0C8
:10117000E6FF01C0E6FF02C0E6FF40C1E6FF41C155
:10118000E6FF87EC11F0036E050EE15E0350000EE2
:10119000E66E010EE66EDAEC00F0E552E552F3CFB2
:1011A000A4F0F4CFA5F08998100EE66E270EE66E37
:1011B000E66AE66A0EEC00F0E552E552E552E552C9
:1011C00081B2FED70CEC01F0230EE66E73EC00F05A
:1011D000E5523A0EE66E73EC00F0E552000EE66E54
:1011E000E66AF1EC11F0E552E5529C0EB16EA09268
:1011F000A192B1800001A26BA36B8998500EE66E9C
:10120000C30EE66EE66AE66A0EEC00F0E552E552C1
:10121000E552E5520001BA6BBB6BBC6BBD6BAA6BB0
:10122000AB6BAC6BAD6B000EE66EE66A0DEC12F0CC
:10123000E552E552898689968986CD809EA012D096
:10124000AA0EE96E000EEA6E0001BA51EE24BA6FE2
:10125000BB51EE20BB6FBC51EE20BC6FBD51EE20E8
:10126000BD6F9E90A1A20DD0A1920001A22B000EF5
:10127000A323320ED880A255000EA35502E289881E
:1012800002D081B0DBD7B190000197A510D0AA0E93
:10129000E96E000EEA6EBA51EE24BA6FBB51EE2031
:1012A000BB6FBC51EE20BC6FBD51EE20BD6F000E78
:1012B000E66E010EE66EBAC0E6FFBBC0E6FFBCC03C
:1012C000E6FFBDC0E6FF6FEC0FF0006E060EE15EBC
:1012D0000050000EE66E010EE66EDAEC00F0E5520C
:1012E000E552F3CFA4F0F4CFA5F00CEC01F0F00E32
:1012F000E66E490EE66E020EE66EE66A0EEC00F051
:10130000E552E552E552E5520001A26BA36BBE6BBC
:10131000BF6BC06BC16BC26B240EC36FF40EC46F86
:10132000C56BBA6BBB6BBC6BBD6BAA6BAB6BAC6BB1
:10133000AD6BD6DD000197A544D2AA0EE96E000E72
:10134000EA6EBA51EE24BA6FBB51EE20BB6FBC51AE
:10135000EE20BC6FBD51EE20BD6FBA0EE96E000EDF
:10136000EA6EEE50BE5DEE50BF59EE50C059EE50E1
:10137000C15908E2BAC0BEF0BBC0BFF0BCC0C0F0EB
:10138000BDC0C1F0BA0EE96E000EEA6EC251EE5C4D
:10139000C351EE58C451EE58C551EE5808E2BAC0D8
:1013A000C2F0BBC0C3F0BCC0C4F0BDC0C5F0E66AAB
:1013B000E66AA2C000F0A3C001F0090ED880005672
:1013C000000E015600C0E6FF01C0E6FFB9EC01F0D7
:1013D000E552E552E552E552090EE66E73EC00F077
:1013E000E552000EE66E010EE66EBAC0E6FFBBC027
:1013F000E6FFBCC0E6FFBDC0E6FF6FEC0FF0006E7D
:10140000060EE15E0050000EE66E010EE66EDAECAE
:1014100000F0E552E552F3CFA4F0F4CFA5F0BA0EF8
:10142000E96E000EEA6E0001B251EE24B26FB351C4
:10143000EE20B36FB451EE20B46FB551EE20B56F0E
:10144000A22B000EA323090ED880A255000EA3558F
:1014500001E3B3D10CEC01F0B2C01CF0B3C01DF03D
:10146000B4C01EF0B5C01FF010EC0CF01DC000F0B1
:101470001EC001F01FC002F020C003F0226A236AE0
:10148000200E246E410E256E00C01DF001C01EF01E
:1014900002C01FF003C020F0C2EC0CF01DC0CAF067
:1014A0001EC0CBF01FC0CCF020C0CDF0B2C0B6F053
:1014B000B3C0B7F0B4C0B8F0B5C0B9F00A0E216E31
:1014C000226A236A246AB6C01CF0B7C01DF0B8C0F7
:1014D0001EF0B9C01FF0AEEC11F01CC0B6F01DC07C
:1014E000B7F01EC0B8F01FC0B9F089B83DD06F0E7C
:1014F000046E120E056E030E066E3A0E076ECAC01B
:1015000022F0CBC023F0CCC024F0CDC025F004C025
:101510001DF005C01EF006C01FF007C020F015EC3E
:101520000DF01DC000F01EC001F01FC002F020C071
:1015300003F0BC0E226E740E236E130E246E3E0E4C
:10154000256E00C01DF001C01EF002C01FF003C0D8
:1015500020F02BEC0CF01DC0C6F01EC0C7F01FC061
:10156000C8F020C0C9F03CD0180E046EB40E056E51
:10157000900E066E380E076ECAC022F0CBC023F064
:10158000CCC024F0CDC025F004C01DF005C01EF075
:1015900006C01FF007C020F015EC0DF01DC000F0D4
:1015A0001EC001F01FC002F020C003F00A0E226E20
:1015B000D70E236E230E246E3D0E256E00C01DF047
:1015C00001C01EF002C01FF003C020F02CEC0CF094
:1015D0001DC0C6F01EC0C7F01FC0C8F020C0C9F0B3
:1015E000000EE66E010EE66EB6C0E6FFB7C0E6FF7F
:1015F000B8C0E6FFB9C0E6FF6FEC0FF0006E060E54
:10160000E15E00502A0EE66E73EC00F0E552000E2B
:10161000E66E010EE66EDAEC00F0E552E552F3CF2D
:10162000A4F0F4CFA5F0090EE66E73EC00F0E552DD
:10163000030EE66E000EE66E010EE66EC6C0E6FF15
:10164000C7C0E6FFC8C0E6FFC9C0E6FFB8EC02F0BD
:10165000006E070EE15E0050000EE66E010EE66EB3
:10166000DAEC00F0E552E552F3CFA4F0F4CFA5F0A8
:10167000200EE66E73EC00F0E55289B806D06E0ECF
:10168000E66E73EC00F0E55205D0750EE66E73EC75
:1016900000F0E552460EE66E73EC00F0E552090EDE
:1016A000E66E73EC00F0E552C20EE96E000EEA6ED3
:1016B000EE500001BE5D086EEE50BF59096EEE504F
:1016C000C0590A6EEE50C1590B6E08C01CF009C01B
:1016D0001DF00AC01EF00BC01FF010EC0CF01DC076
:1016E00004F01EC005F01FC006F020C007F0226AFB
:1016F000236AC80E246E420E256E04C01DF005C07C
:101700001EF006C01FF007C020F015EC0DF01DC044
:1017100000F01EC001F01FC002F020C003F0CAC0DC
:1017200022F0CBC023F0CCC024F0CDC025F000C007
:101730001DF001C01EF002C01FF003C020F0C2EC7B
:101740000CF01DC0C6F01EC0C7F01FC0C8F020C0FE
:10175000C9F02B0EE66E73EC00F0E5522D0EE66E2E
:1017600073EC00F0E552020EE66E000EE66E010E1E
:10177000E66EC6C0E6FFC7C0E6FFC8C0E6FFC9C048
:10178000E6FFB8EC02F0006E070EE15E0050000EBE
:10179000E66E010EE66EDAEC00F0E552E552F3CFAC
:1017A000A4F0F4CFA5F0250EE66E73EC00F0E55240
:1017B0000001B26BB36BB46BB56B0CEC01F00001C4
:1017C0009795A80EE66E610EE66EE66AE66A0EEC86
:1017D00000F0E552E552E552E55200010A0EA25D25
:1017E000000EA35901E2A5D50CEC01F00001A26B9B
:0617F000A36BB8D4120047
:0A17F600279E08D0279E1FAE05D0E5
:101800001E6C1F1EE86A1F22278E1FC019F01EC003
:1018100018F02B6A2A6A8E0E1A6E1B6A6BEF0EF096
:10182000279E0CD0279E1FAE09D01C6C1D1E1E1EAD
:101830001F1EE86A1D221E221F22278E1FC019F0BC
:101840001EC018F01DC02BF01CC02AF09E0E1A6E90
:101850001B6A6BEF0EF0257E276AA7EC0EF0BFEC3B
:101860000EF027B64FEF0EF027A20AD027AA03D01A
:1018700027BE4FEF0EF027A45BEF0EF058EF0EF0EF
:1018800027AA05D027AC5BEF0EF058EF0EF027A08B
:101890000AD027A808D027BE04D027A402D064EF1E
:1018A0000EF068EF0EF02A6A1B6A2550205C296E44
:1018B00010E31DC02BF01EC018F01FC019F020C08F
:1018C00028F022C01DF023C01EF024C01FF0273ACC
:1018D00009D022C02BF023C018F024C019F025C075
:1018E00028F0296C279E27BC278E28C01AF027B025
:1018F00097EF0EF01A0E296097EF0EF01A6A206A21
:1019000027A408D01D6C1E1E1F1E201EE86A1E2262
:101910001F22202227AC08D02B6C181E191E1A1E5D
:10192000E86A182219221A221C6A295207E0203478
:101930001F321E321D321C32292EF9D71D502B2684
:101940001E5018221F50192220501A221CC02AF0A3
:10195000279E1AAE0BD02A6C2B1E181E191E1A1E9B
:10196000E86A2B22182219221A22278E1AA006D0E2
:10197000D880193218322B322A32282A28C01AF07D
:101980006BEF0EF0276AA7EC0EF0BFEC0EF027B657
:101990004FEF0EF027A205D027BA4FEF0EF056EF0B
:1019A0000EF027BA62EF0EF027A005D027B84FEF50
:1019B0000EF062EF0EF027B856EF0EF01B6A7F0EA6
:1019C00020241A6EE86A1B2225501A5EE86A1B5A08
:1019D0001A0E286E206A2A6A2B6A186A196A22501F
:1019E0001D5E23501E5A24501F5A000E205A09E72C
:1019F00022501D2623501E2224501F22000E20227A
:101A000001D02A8AD8901D361E361F362036D8902F
:101A10002A362B3618361936282EE1D71F501E10BD
:101A20001D10D8A42A8A6BEF0EF0276AA7EC0EF0DF
:101A3000BFEC0EF027B64FEF0EF027A205D027B867
:101A40004FEF0EF056EF0EF027AA05D027B04FEF5C
:101A50000EF056EF0EF027B002D027A802D062EFAA
:101A60000EF01B6A255020241A6EE86A1B227E0E97
:101A70001A5EE86A1B5A2A6A2B6A186A196A245085
:101A80001F02F4CF19F0F3CF18F023501F02F350C8
:101A90002B26F4501822000E192224501E02F35057
:101AA0002B26F4501822000E192222501F02F35048
:101AB0002A26F4502B22000E1822192223501E022F
:101AC000F3502A26F4502B22000E182219222450FB
:101AD0001D02F3502A26F4502B22000E1822192240
:101AE00022501E02F4502A26000E2B221822192200
:101AF00023501D02F4502A26000E2B2218221922F0
:101B00006BEF0EF0276AA7EC0EF027B68CEF0DF006
:101B100027A20ED027B405D07F0E1F6EFF0E1E6EBB
:101B20001FD0800E1F6E1E6A1BD01F6A1E6A18D03F
:101B300027B0FBD78F0E2060EDD77E0E2064F5D73F
:101B40008E0E205C05E0D8901F321E32202AF8D776
:101B500027A406D01E6C1F1EE86A1F221FAEE5D701
:101B60001200276AA7EC0EF027B6BBEF0DF027A2F4
:101B70000FD027B407D07F0E1F6EFF0E1E6E1D6E96
:101B80001C6E25D0800E1F6E01D01F6A000EF6D786
:101B900027B0FBD71C6A9F0E2060EBD77E0E206417
:101BA000F4D79E0E205C07E0D8901F321E321D3203
:101BB0001C32202AF6D727A40AD01C6C1D1E1E1E1C
:101BC0001F1EE86A1D221E221F221FAEDED7120032
:101BD000FAEC0DF027B6000C27B0000C27B4000C6F
:101BE000010CFAEC0DF027B6000C27B0000C27A46E
:101BF000000C010C276AA7EC0EF0BFEC0EF027B624
:101C0000120027AE08D027A004D027A802D0278032
:101C10001200279012002550205C0BE124501F5C1D
:101C200008E123501E5C05E122501D5C02E1278083
:101C30001200D8A002D0278E10D0205025C020F04E
:101C4000256E1F5024C01FF0246E1E5023C01EF0AE
:101C5000236E1D5022C01DF0226E2550205C10E026
:101C6000FF0F09E0279027B403D027AE2784120086
:101C700027AE27941200252AD8902432233222320C
:101C800022501D5E23501E5A24501F5A1FBEEAD7F1
:101C9000D8901D361E361F36202EF8D7C8D77F0E97
:101CA000206EFF0E1F6E1E6E1D6E12007F0E27BE71
:101CB000FF0E206E02D07F0E206E800E1F6E1E6AF9
:101CC0001D6AF3D727AE04D0800E206E1F6AF7D7A7
:101CD000206A1F6AF4D7195018102B102A10F8E048
:101CE0001BBEF0D719BE0CD01A501B10EBE0D890D9
:101CF0002A362B36183619361A06D8A01B06F2D704
:101D00001B50D4E11A28D2E02AAE11D07F0E2A143B
:101D100002E12BA00CD02B2AE86A1822192207E333
:101D2000D880193218322B321A2A1A28BFE01A50DA
:101D3000C9E02BC01DF018C01EF019341F6E1A30F8
:101D4000206E1F32209E27BE208E55EF0EF01F36CC
:101D5000203602E32784277E06E12780206A1F6A57
:101D60001E6A1D6A1200202803E0D8801F3212006C
:101D7000D8901F3202E127821200278612002436F3
:101D8000253602E3278C277E06E12788256A246A08
:101D9000236A226A1200252803E0D8802432120028
:0A1DA000D8902432EAE1278A1200ED
:061DAA00D9CFE6FFDACFFD
:101DB000E6FFFA0EE3CFD9FFFB0EE3CFDAFFFD0E0D
:101DC000E35209E72D0EDE6EFC0EE31EE32AFD0E44
:101DD000D8B4E306E31EE652E652E652FD0EE124D5
:101DE000E76EFF0EE220E46EE652F70EE3CFE6FF69
:101DF000F70EE3CFE6FF45EC0FF0F90EE124E96EB4
:101E0000FF0EE220EA6E35EC0FF00AE132EC0FF043
:101E100009E135EC0FF008E132EC0FF007E108D0F2
:101E200040EC0FF03BEC0FF040EC0FF03BEC0FF010
:101E300040EC0FF0DE6AF90EE126FF0EE222FF0E03
:101E4000E3CFDAFFE552FF0EE3CFD9FFE552FC0EF8
:101E5000E124E96EFF0EE220EA6EEECFF3FFEFCF52
:101E6000F4FF1200EF380F0B1200EF500F0B02E1DE
:101E7000EE52D8841200EF380F0B300FDE6E1200D6
:101E8000EE500F0B300FDE6E1200FC0EE3CFE9FFB9
:101E9000FD0EE3CFEAFF100EE66EEE6AEE6AEF6A21
:101EA000D890FD0EE336FE0EE336ED36ED36EF3616
:101EB000FF0EE30609E066EC0FF0EE5266EC0FF061
:101EC000EE5266EC0FF0EDD7E56E1200030EEF2434
:101ED000E8B6EF6E300EEF24E8BEEF6E000CD9CFFF
:101EE000E6FFDACFE6FFF80EE3CFD9FFF90EE3CF36
:101EF000DAFFE652E652E652E652E652FB0EE124E3
:101F0000E76EFF0EE220E46EE652F30EE3CFE6FF4B
:101F1000F30EE3CFE6FFF30EE3CFE6FFF30EE3CFDE
:101F2000E6FFF4EC0FF0F50EE124E96EFF0EE2207F
:101F3000EA6EE1EC0FF019E1E4EC0FF018E1E1ECEE
:101F40000FF017E1E4EC0FF016E1E1EC0FF015E112
:101F5000E4EC0FF014E1E1EC0FF013E1E4EC0FF02E
:101F600012E1E1EC0FF011E112D0EAEC0FF0EFEC2E
:101F70000FF0EAEC0FF0EFEC0FF0EAEC0FF0EFEC03
:101F80000FF0EAEC0FF0EFEC0FF0EAEC0FF0EFECF3
:101F90000FF0DE6AF50EE126FF0EE222FF0EE3CF20
:101FA000DAFFE552FF0EE3CFD9FFE552FA0EE12446
:101FB000E96EFF0EE220EA6EEECFF3FFEFCFF4FF03
:101FC0001200EF380F0B1200EF500F0B02E1EE5230
:101FD000D8841200EF380F0B300FDE6E1200EE5077
:101FE0000F0B300FDE6E1200FA0EE3CFE9FFFB0E8F
:101FF000E3CFEAFF200EE66EEE6AEE6AEE6AEE6A64
:10200000EF6AD890FB0EE336FC0EE336FD0EE336A6
:10201000FE0EE336ED36ED36ED36ED36EF36FF0EDD
:10202000E3060FE023EC10F0EE5223EC10F0EE523A
:1020300023EC10F0EE5223EC10F0EE5223EC10F0F3
:10204000E1D7E56E1200030EEF24E8B6EF6E300E16
:08205000EF24E8BEEF6E000C66
:082058002E2E2E00506F727451
:1020600020636F6D6D203338343030206F757665A6
:102070007274200D0A00696E746572666163652072
:1020800049434D373535352C20513D32304D687A36
:10209000202C52656C6169732047616D6D652C2041
:1020A0004250207374617274200D0A004331383A33
:1020B000203138465F4361706163696D5F49434D0C
:1020C000373535355F434350315F32304D687A5F85
:1020D00052533233325F3132313232362E630D0A8F
:1020E000004F4B204D657375726520436170612010
:1020F0005A45524F3D313030203A200050524F4225
:102100004C454D4521204D657375726520436170C6
:10211000615A65726F20313030704620494E5354F9
:1021200041424C452120323837202B2D35203A2092
:1021300000496E7365726572204378206574206172
:1021400070707579657220737572204250207374B7
:102150006172742000313846204361706163696D9B
:102160006574657220002049434D37353535202090
:102170002020202020200020204D504C4142204390
:102180003138202020202000203235206465632053
:10219000203230313120202000204361706163699A
:1021A0007465204E616E6F462000204F7665722068
:1021B0002121212020202020202000204D6F796522
:1021C0006E6E65203130206D657320002043617094
:1021D000616369746520656E207546200020537424
:1021E0006162696C69746520202020202000204DE8
:0F21F0006573757265202020202020202020009C
:102200000E0EF66E000EF76E000EF86E000109005D
:10221000F550DB6F0900F550DC6F03E1DB6701D09F
:102220003DD00900F550D66F0900F550D76F090071
:10223000F550D86F09000900F550E96E0900F55016
:10224000EA6E090009000900F550D96F0900F55040
:10225000DA6F09000900F6CFDDF0F7CFDEF0F8CF36
:10226000DFF0D6C0F6FFD7C0F7FFD8C0F8FF0001F7
:10227000D95302E1DA5307E00900F550EE6ED907B1
:10228000F8E2DA07F9D7DDC0F6FFDEC0F7FFDFC0FE
:0E229000F8FF0001DB07000EDC5BBFD7120079
:02229E001C50D2
:1022A0002102F3CF18F0F4CF19F02202F3501926CF
:1022B000000EF4201A6E1C502302F3501A26000E52
:1022C000F4201B6E1C502402F3501B261D502102CB
:1022D000F3501926F4501A22000E1B221D50220220
:1022E000F3501A26F4501B221D502302F3501B26D4
:1022F0001E502102F3501A26F4501B221E502202B7
:0E230000F3501B261F502102F3501B26120023
:02230E00FB0EC4
:10231000E3CFF6FFFC0EE3CFF7FFFD0EE3CFF8FFB0
:10232000FE0EE3CFE9FFFF0EE3CFEAFFE9CFF3FFB5
:10233000EACFF4FF0900F5CFEFFFEE66FBD71200FE
:10234000FE0EE3CFE9FFFF0EE3CFEAFFF36AF46A84
:0C235000EE5203E0F34AF42AFBD712001F
:04235C001B6A1A6A74
:10236000196A186A200EE76ED8901C361D361E3684
:102370001F36183619361A361B362150185C225073
:10238000195823501A5824501B5809E32150185E3D
:102390002250195A23501A5A24501B5A1C2AE72E2D
:0423A000E4D712006C
:0C23A400D9CFE6FFDACFE6FFE1CFD9FF8A
:1023B000E2CFDAFFE652F20E0001E017ABAC03D039
:1023C000E091ABB0E081ABB4E085ABB2E087AE505A
:1023D000DF6EDF50E552E552E5CFDAFFE7CFD9FFF8
:0223E0001200E9
:0E23E200D9CFE6FFDACFE6FFE1CFD9FFE2CF99
:1023F000DAFFE652E652FC0EDBCFDEFFDBCFDDFF7D
:10240000010EDB50B36EDF50B26EE552E552E5527D
:0A241000E5CFDAFFE7CFD9FF120095
:06241A00D9CFE6FFDACF86
:10242000E6FFE1CFD9FFE2CFDAFFE652E652FC0E3B
:10243000DBCFDEFFDBCFDDFF010EDB50CF6EDF50E9
:10244000CE6EE552E552E552E5CFDAFFE7CFD9FF90
:02245000120078
:0E245200D9CFE6FFDACFE6FFE1CFD9FFE2CF28
:10246000DAFFACAC04D0AC900001E0B3AC80FD0E60
:10247000DB50AD6EE552E5CFDAFFE7CFD9FF1200B2
:10248000000EF36E00EE00F0060E01D81200EA60B6
:1024900002D0EE6AFCD7F350E9601200EE6AFCD776
:1024A00015EE00F025EE00F0F86A279C00EC11F024
:0C24B00003EC00F08BEC07F0FBD71200EF
:0424BC00313846323B
:1024C00035325F4361706163696D5F434135353516
:1024D0005F706F6F6C696E672E630D0A20207374D6
:1024E00072696E6720656E2052414D0D000000003C
:1024F0000000000000000000000000000001313278
:1025000033343536373839303132333435000430EE
:1025100030303030303030303030303030303030BB
:102520003030303030300004040404040404040467
:10253000040404040404040404040404040404045B
:1025400004040404040404040404040404040458F7
:10255000205C207620AC20E120FC20312155216632
:1025600021772188219921AA21BB21CC21DD21EECF
:0525700021B31501007C
:020000040030CA
:01000100FA04
:01000200F409
:01000300FEFE
:01000600FBFE
:00000001FF
